:020000040000FA
:100000003B290E088F000F08233C031C0F280F0804
:10001000113C031C0D2805301828093018282430FD
:100020008F020F08113C031C17280A3018280630CD
:100030009100141D41280F08820747284C28532897
:100040005A285F2866286D287228792880288528F4
:100050008C28932898289F28A628AB28B228B9284E
:10006000BE28C528CC28D128D828DF28E428EB28AA
:10007000F228F728FE2805290A29112918291D29FF
:100080002429100882072B292F2933293729110801
:10009000C0389300920069291108C03893001108F4
:1000A000D038920069291108D03893001108C0385F
:1000B000920069291108D03893009200692911082B
:1000C000D03893001108E038920069291108E0380F
:1000D00093001108D038920069291108E038930084
:1000E000920069291108E03893001108F038920055
:1000F00069291108F03893001108E0389200692945
:100100001108F0389300920069291108F038930023
:100110001108B038920069291108B038930011080D
:10012000F038920069291108B038930092006929CB
:100130001108B0389300110870389200692911082D
:10014000703893001108B03892006929110870388E
:100150009300920069291108703893001108303813
:100160009200692911083038930011087038920004
:100170006929110830389300920069291108303834
:1001800093001108703892006929110870389300A3
:1001900011083038920069291108703893009200D4
:1001A00069291108703893001108B0389200692944
:1001B0001108B038930011087038920069291108AD
:1001C000B0389300920069291108B03893001108E3
:1001D000F038920069291108F03893001108B038FE
:1001E000920069291108F0389300920069291108DA
:1001F000F03893001108E038920069291108E038BE
:1002000093001108F038920069291108E038930032
:10021000920069291108E03893001108D038920043
:1002200069291108D03893001108E0389200692933
:100230001108D0389300920069291108D038930032
:100240001108C038920069291108C03893001108BC
:10025000D03892006929953093009200692969305D
:100260009300920069296A309300920069299630C0
:10027000930092006929732101283B2914089506EF
:10028000151C6229141C6229141D5429941C4E2922
:100290008E038E1F622947308E0062298E0A0E0857
:1002A000473C031C8E016229941C5C299003901F1B
:1002B0006229033090006229900A1008033C031C55
:1002C0009001622914089500012812088600000098
:1002D00000001308860000000508150603196529AB
:1002E000150694003E298230831681008312860110
:1002F000003083168600831285010730831685003F
:10030000831200308A000C3084008001840A0408C3
:10031000503C031D852900308E000508940095008F
:0603200000308B00080014
:02400E00F13F80
:00000001FF
